BL51 BANKED LINKER/LOCATER V6.22.2.0                                                    02/02/2023  15:35:32  PAGE 1


BL51 BANKED LINKER/LOCATER V6.22.2.0, INVOKED BY:
C:\KEIL_V5\C51\BIN\BL51.EXE .\Release\system_FE81001.obj, .\Release\STARTUP.obj, .\Release\main.obj TO .\Release\Sample_
>> DrvFMC REGFILE (.\Release\Sample_DrvFMC.ORC) PRINT (.\Sample_DrvFMC.m51) RAMSIZE (256) CODE (0X0000-0X1FFF) XDATA (0X
>> 8000-0X87FF)


MEMORY MODEL: SMALL


INPUT MODULES INCLUDED:
  .\Release\system_FE81001.obj (SYSTEM_FE81001)
  .\Release\STARTUP.obj (?C_STARTUP)
  .\Release\main.obj (MAIN)
  C:\KEIL_V5\C51\LIB\C51S.LIB (?C_IBP)


LINK MAP OF MODULE:  .\Release\Sample_DrvFMC (SYSTEM_FE81001)


            TYPE    BASE      LENGTH    RELOCATION   SEGMENT NAME
            -----------------------------------------------------

            * * * * * * *   D A T A   M E M O R Y   * * * * * * *
            REG     0000H     0008H     ABSOLUTE     "REG BANK 0"
            DATA    0008H     0008H     UNIT         ?DT?MAIN?MAIN
            DATA    0010H     0008H     UNIT         ?DT?_RE_FLASH?MAIN
            DATA    0018H     0005H     UNIT         ?DT?_RE_INFORMATION_BLOCK?MAIN
            DATA    001DH     0003H     UNIT         ?DT?_WR_INFORMATION_BLOCK?MAIN
            DATA    0020H     0002H     UNIT         ?DT?DELAY?MAIN
            DATA    0022H     0001H     UNIT         ?C?LIB_DATA
            IDATA   0023H     0001H     UNIT         ?STACK

            * * * * * * *   C O D E   M E M O R Y   * * * * * * *
            CODE    0000H     0003H     ABSOLUTE     
            CODE    0003H     0092H     UNIT         ?PR?MAIN?MAIN
            CODE    0095H     004FH     UNIT         ?PR?_RE_FLASH?MAIN
            CODE    00E4H     004CH     UNIT         ?PR?_RE_INFORMATION_BLOCK?MAIN
            CODE    0130H     0041H     UNIT         ?PR?_WR_INFORMATION_BLOCK?MAIN
            CODE    0171H     001DH     UNIT         ?C_C51STARTUP
            CODE    018EH     001CH     UNIT         ?PR?DELAY?MAIN
            CODE    01AAH     0001H     UNIT         ?PR?SYSTEMINIT?SYSTEM_FE81001



OVERLAY MAP OF MODULE:   .\Release\Sample_DrvFMC (SYSTEM_FE81001)


SEGMENT
  +--> CALLED SEGMENT
---------------------
?C_C51STARTUP
  +--> ?PR?MAIN?MAIN

?PR?MAIN?MAIN
  +--> ?PR?_WR_INFORMATION_BLOCK?MAIN
  +--> ?PR?_RE_INFORMATION_BLOCK?MAIN
  +--> ?PR?_RE_FLASH?MAIN
  +--> ?PR?DELAY?MAIN
BL51 BANKED LINKER/LOCATER V6.22.2.0                                                  02/02/2023  15:35:32  PAGE 2





SYMBOL TABLE OF MODULE:  .\Release\Sample_DrvFMC (SYSTEM_FE81001)

  VALUE           TYPE          NAME
  ----------------------------------

  -------         MODULE        SYSTEM_FE81001
  C:0000H         SYMBOL        _ICE_DUMMY_
  C:01AAH         PUBLIC        SystemInit
  -------         PROC          SYSTEMINIT
  C:01AAH         LINE#         38
  C:01AAH         LINE#         39
  C:01AAH         LINE#         41
  -------         ENDPROC       SYSTEMINIT
  -------         ENDMOD        SYSTEM_FE81001

  -------         MODULE        ?C_STARTUP
  C:0171H         SEGMENT       ?C_C51STARTUP
  I:0023H         SEGMENT       ?STACK
  C:0000H         PUBLIC        ?C_STARTUP
  D:00E0H         SYMBOL        ACC
  D:00F0H         SYMBOL        B
  D:0083H         SYMBOL        DPH
  D:0082H         SYMBOL        DPL
  N:0001H         SYMBOL        IBPSTACK
  N:0100H         SYMBOL        IBPSTACKTOP
  N:0080H         SYMBOL        IDATALEN
  C:0174H         SYMBOL        IDATALOOP
  N:0000H         SYMBOL        PBPSTACK
  N:0100H         SYMBOL        PBPSTACKTOP
  N:0000H         SYMBOL        PDATALEN
  N:0000H         SYMBOL        PDATASTART
  N:0000H         SYMBOL        PPAGE
  N:0000H         SYMBOL        PPAGEENABLE
  D:00A0H         SYMBOL        PPAGE_SFR
  D:0081H         SYMBOL        SP
  C:0171H         SYMBOL        STARTUP1
  N:0000H         SYMBOL        XBPSTACK
  N:0000H         SYMBOL        XBPSTACKTOP
  N:0800H         SYMBOL        XDATALEN
  C:017FH         SYMBOL        XDATALOOP
  N:8000H         SYMBOL        XDATASTART
  C:0000H         LINE#         126
  C:0171H         LINE#         133
  C:0173H         LINE#         134
  C:0174H         LINE#         135
  C:0175H         LINE#         136
  C:0177H         LINE#         140
  C:017AH         LINE#         141
  C:017CH         LINE#         145
  C:017EH         LINE#         147
  C:017FH         LINE#         148
  C:0180H         LINE#         149
  C:0181H         LINE#         150
  C:0183H         LINE#         151
BL51 BANKED LINKER/LOCATER V6.22.2.0                                                  02/02/2023  15:35:32  PAGE 3


  C:0185H         LINE#         170
  C:0188H         LINE#         185
  C:018BH         LINE#         196
  -------         ENDMOD        ?C_STARTUP

  -------         MODULE        MAIN
  C:0000H         SYMBOL        _ICE_DUMMY_
  D:0090H         PUBLIC        P1
  D:00B0H         PUBLIC        P3
  C:0095H         PUBLIC        _RE_flash
  D:00A8H         PUBLIC        IE
  C:018EH         PUBLIC        delay
  C:00E4H         PUBLIC        _RE_information_block
  D:00B8H         PUBLIC        IP
  C:0003H         PUBLIC        main
  C:0130H         PUBLIC        _WR_information_block
  D:0098H         PUBLIC        SCON
  D:0088H         PUBLIC        TCON
  D:00C8H         PUBLIC        T2CON
  D:00D0H         PUBLIC        PSW
  -------         PROC          DELAY
  -------         DO            
  D:0020H         SYMBOL        i
  -------         ENDDO         
  C:018EH         LINE#         35
  C:018EH         LINE#         36
  C:018EH         LINE#         39
  C:01A9H         LINE#         40
  -------         ENDPROC       DELAY
  -------         PROC          MAIN
  -------         DO            
  D:0008H         SYMBOL        RE_data1
  D:000AH         SYMBOL        RE_data2
  D:000CH         SYMBOL        RE_data3
  D:000EH         SYMBOL        RE_data4
  -------         ENDDO         
  C:0003H         LINE#         52
  C:0003H         LINE#         53
  C:0003H         LINE#         57
  C:000EH         LINE#         60
  C:002FH         LINE#         62
  C:0034H         LINE#         63
  C:003AH         LINE#         64
  C:003FH         LINE#         67
  C:004AH         LINE#         69
  C:0053H         LINE#         70
  C:005CH         LINE#         72
  C:0065H         LINE#         73
  C:006EH         LINE#         75
  C:0077H         LINE#         76
  C:0080H         LINE#         79
  C:008FH         LINE#         83
  C:0092H         LINE#         85
  -------         ENDPROC       MAIN
  -------         PROC          _WR_INFORMATION_BLOCK
  D:001DH         SYMBOL        addr
  D:001EH         SYMBOL        dataH
BL51 BANKED LINKER/LOCATER V6.22.2.0                                                  02/02/2023  15:35:32  PAGE 4


  D:001FH         SYMBOL        dataL
  C:0130H         LINE#         88
  C:0136H         LINE#         89
  C:0136H         LINE#         91
  C:013CH         LINE#         94
  C:0142H         LINE#         95
  C:0147H         LINE#         96
  C:014DH         LINE#         97
  C:0153H         LINE#         98
  C:0159H         LINE#         99
  C:016AH         LINE#         100
  C:016AH         LINE#         103
  C:0170H         LINE#         105
  -------         ENDPROC       _WR_INFORMATION_BLOCK
  -------         PROC          _RE_INFORMATION_BLOCK
  D:0018H         SYMBOL        addrL
  -------         DO            
  D:0019H         SYMBOL        infodata
  D:001BH         SYMBOL        data0
  D:001CH         SYMBOL        data1
  -------         ENDDO         
  C:00E4H         LINE#         107
  C:00E6H         LINE#         108
  C:00E6H         LINE#         112
  C:00ECH         LINE#         114
  C:00F2H         LINE#         115
  C:00F7H         LINE#         116
  C:00FDH         LINE#         117
  C:0104H         LINE#         118
  C:010AH         LINE#         119
  C:0111H         LINE#         120
  C:0125H         LINE#         123
  C:012BH         LINE#         124
  C:012FH         LINE#         126
  -------         ENDPROC       _RE_INFORMATION_BLOCK
  -------         PROC          _RE_FLASH
  D:0010H         SYMBOL        addrH
  D:0012H         SYMBOL        addrL
  -------         DO            
  D:0014H         SYMBOL        infodata
  D:0016H         SYMBOL        data0
  D:0017H         SYMBOL        data1
  -------         ENDDO         
  C:0095H         LINE#         127
  C:009DH         LINE#         128
  C:009DH         LINE#         133
  C:00A3H         LINE#         135
  C:00AAH         LINE#         136
  C:00B1H         LINE#         137
  C:00B7H         LINE#         138
  C:00BEH         LINE#         139
  C:00C4H         LINE#         140
  C:00CBH         LINE#         141
  C:00DFH         LINE#         143
  C:00E3H         LINE#         144
  -------         ENDPROC       _RE_FLASH
  -------         ENDMOD        MAIN
BL51 BANKED LINKER/LOCATER V6.22.2.0                                                  02/02/2023  15:35:32  PAGE 5



  -------         MODULE        ?C_IBP
  D:0022H         PUBLIC        ?C_IBP
  -------         ENDMOD        ?C_IBP



FUNCTION REGISTER MASKS


FUNCTION . . . . . . . . REG MASK
---------------------------------

DELAY. . . . . . . . . . @0xf000
SYSTEMINIT . . . . . . . @0x8000
_RE_FLASH. . . . . . . . @0xe30f
_RE_INFORMATION_BLOCK. . @0xe30f
_WR_INFORMATION_BLOCK. . @0xe303

*** WARNING L16: UNCALLED SEGMENT, IGNORED FOR OVERLAY PROCESS
    SEGMENT: ?PR?SYSTEMINIT?SYSTEM_FE81001

Program Size: data=36.0 xdata=0 code=427
LINK/LOCATE RUN COMPLETE.  1 WARNING(S),  0 ERROR(S)
